:1000000019C033C032C055C030C02FC02EC02DC063
:100010002CC02BC02AC029C028C027C026C025C09C
:1000200024C023C022C021C020C01FC01EC01DC0CC
:100030001CC01BC011241FBECFEFCDBFDFE3DEBF4E
:100040001FE3A0E8BFE3E8E6F4E002C005900D92EC
:10005000A438B107D9F72FE3A4E8BFE301C01D928C
:10006000AE38B207E1F7EED0E8C1CACF81B1857FE3
:1000700081B910922C0A10922D0A089581B18A60DC
:1000800081B98FEF90E080932C0A90932D0A089508
:10009000E0E0FAE083E481838FEF90E086A397A30A
:1000A00081E08083089590E080932C0A90932D0A3C
:1000B00008958F939F9381E080930904109905C060
:1000C00098ED94BF80934100FFCF9F918F91189539
:1000D000CF93DF93811549F01092893F10928A3FA8
:1000E0008CE08093813F1092883FC091893FD091EE
:1000F0008A3F2196C093893FD0938A3FE091813F08
:10010000E53170F4F0E0E15EFD4F0994AFDF6997EF
:1001100038F01092893F10928A3F82E08093813FAD
:10012000DF91CF91089581B18A6081B92597C0F39D
:100130001092893F10928A3F85E0F0CF97DF2A978F
:1001400078F31092893F10928A3F87E0E7CF81B120
:100150008A6081B9259720F31092893F10928A3FD7
:100160008AE0DCCF83DF6997D8F21092893F109242
:100170008A3F8CE0D3CF8FEF90E080932C0A90934E
:100180002D0A259768F21092893F10928A3F8EE0DF
:10019000C5CF6CDF2A9720F21092893F10928A3FD8
:1001A00080E1BCCF8FEF90E080932C0A90932D0AD2
:1001B000259708F4B5CF1092893F10928A3F82E1CB
:1001C000ADCF54DF699708F4ABCF1092893F1092FE
:1001D0008A3F8091883F8F5F8093883F833060F0B3
:1001E0001092883F84E19ACF49DF699708F498CF4D
:1001F0001092893F10928A3F1092813F91CF3ECF5B
:100200008091873F9091803F890F8093873F84360C
:10021000A8F084E68093873F8FEF8093803F8091A2
:10022000873F2FEF829FC001112464E670E0F2D077
:10023000772760932C0A70932D0A08958A3079F7F6
:1002400081E0EBCF80E380930104809306048091EA
:100250005000897F809350001092400A80910006E0
:100260008E7F80930006809170068E7F809370064B
:100270001092060810921308109219081092200884
:100280008EEC80B905DF009888E080931004EEDEE4
:1002900081B1806C81B91091823F1092843F10929D
:1002A000853F01E0C3E0D0E09BE0F92E82B1817090
:1002B000282F2027811115C080918C3F90918D3F70
:1002C0008F3F980741F0019680938C3F90938D3F2C
:1002D0008436910508F18091823F80278093823F88
:1002E0001BC080918B3F811599F080918C3F90913C
:1002F0008D3F05978F35910558F48091843F9091FB
:10030000853F0196BE0172D08093843F9093853FD4
:1003100010928C3F10928D3F20938B3F2093863F0D
:100320008091863F811509F444C0A8DE8091823F08
:10033000811709F440C01091823F8AE0E82E96DED2
:1003400083E294EF0197F1F700C0000097DE83E2AB
:1003500094EF0197F1F700C0000088DEEA9479F786
:100360009FE724E83EE1915020403040E1F700C093
:100370000000F092100480915000897F8260809389
:10038000500080915000816080935000789488954F
:100390008091500081608093500083ED90E301973D
:1003A000F1F700C00000809150008E7F80935000D4
:1003B0007DCF5CDEBBCF8091823F811549F3809178
:1003C000863F8111E5CF8091843F9091853F8130B8
:1003D000910541F08230910539F0892BC9F680E012
:1003E00077DED6CF0DDFD4CF49DED2CFAA1BBB1B21
:1003F00051E107C0AA1FBB1FA617B70710F0A61B25
:10040000B70B881F991F5A95A9F780959095BC0145
:10041000CD01089597FB072E16F4009406D077FDC2
:1004200008D0E4DF07FC05D03EF4909581959F4FFE
:100430000895709561957F4F0895F894FFCF66CE2B
:100440006FCE71CE6DCE6CCE79CE6ACE80CE68CEB8
:1004500067CE88CE65CE8FCE63CE9BCE61CEA2CE48
:080460005FCEAFCE5DCEC0CE31
:04046800010201008C
:00000001FF
